:0809540002080096C180C101F8
:10088C00758911E4F58A758CDCC28DD28CD2A9D213
:10089C00AF7590FF120912A2019290120912A201D7
:1008AC009291120912A2019292120912A201929330
:1008BC00120912A2019294120912A2019295120924
:1008CC0012A2019296120912A2019297120912A277
:1008DC00009297120912A2009296120912A200928B
:1008EC0095120912A2009294120912A2009293126C
:1008FC000912A2009292120912A2009291120912EC
:06090C00A2009290808E13
:10091200E4FFFEC28FC28EE4F58B758DDCD28E3081
:100922008FFDC28EC28F0FBF00010EEF64964E7014
:01093200E2E2
:0109330022A1
:03000B00020934B3
:10093400C0E0758A00758CDCC28DE509150970026A
:100944001508E50945087005F508750996D0E032E3
:03000000020800F3
:0C080000787FE4F6D8FD758120020847DF
:10080C0002088CE493A3F8E493A34003F68001F26E
:10081C0008DFF48029E493A3F85407240CC8C333ED
:10082C00C4540F4420C8834004F456800146F6DFBC
:10083C00E4800B0102040810204080900954E47EEF
:10084C00019360BCA3FF543F30E509541FFEE493B1
:10085C00A360010ECF54C025E060A840B8E493A378
:10086C00FAE493A3F8E493A3C8C582C8CAC583CAA3
:10087C00F0A3C8C582C8CAC583CADFE9DEE780BE5B
:01095C00009A
:00000001FF
